:020000040000FA
:02000000CA280C
:08000800831203138B13831212
:100010000313AE00831203138C1C29288C10831247
:100020000313910183120313BE0B242883160313B9
:100030008C1083120313121183120313AD14831255
:1000400003132E088B170900831203132E088B1736
:1000500009008316031387108312031310108312F1
:1000600003130C10831203132D183B282D14831235
:10007000031387144228831203132D1083120313D2
:1000800087104228831203132008831203138F0062
:10009000831203132108831203138E0083120313A8
:1000A0002E088312031310148B17090083120313F5
:1000B0002B0883120313AC003330AC02031C08007E
:1000C00083120313AB01AB0A08006400831203130D
:1000D0009F01831203138701831603138701831281
:1000E000031386018316031386018312031385010C
:1000F000831203179E01831203179F0183160313B4
:1001000016308500831603138113831603131630EC
:100110009500080083120313053090008316031323
:100120000C14831203130C1083120313C0308B00C2
:1001300083120313FF309200831603138C10831273
:1001400003138C10FF308316031392000800AF01D5
:100150006400B00BA8280800831603130030900039
:100160000800831603136B308F00080083160313F7
:100170005B308F000800831603134B308F0008009C
:10018000831603130B308F000800831603132B30E4
:100190008F0008008A20C520BE22BE22AC20D922B2
:1001A00097223623652083120313BD238312031382
:1001B0000F30B1005620B1208A1500288312031396
:1001C0000F30B100BB2056208B1384238B13B12337
:1001D0008B17B1208B1764008B1783120313AD1894
:1001E00032218312031305190A298B138312031377
:1001F000AB0A2B0883120313AC003330AC02031993
:1002000003298A15002883120313AB01AB0A8B1351
:100210008A150028831203138518EB288B13831289
:100220000313AB0B142917298B138A15002883128B
:1002300003133230AB008A150028831203133108F0
:1002400083120313B2000230B20283120313031DA0
:1002500008008717C020C2228713B120831203131E
:10026000B101080083120313051E08008312031353
:10027000AD10831203132B0883120313B800B901C6
:10028000EF2283120313360883120313BF00562193
:10029000F621F621F621F621F621F6218312031329
:1002A000370883120313BF0056210800831203137B
:1002B0003F0883120313C0000130C002031D6629EA
:1002C0000822FF21FF21FF21FF21080083120313D1
:1002D0003F0883120313C0000230C002031D7629B9
:1002E00008220822FF21FF21FF21080083120313A7
:1002F0003F0883120313C0000330C002031D862988
:10030000082208220822FF21FF210800831203137C
:100310003F0883120313C0000430C002031D962956
:100320000822082208220822FF2108008312031352
:100330003F0883120313C0000530C002031DA62925
:100340000822082208220822082208008312031328
:100350003F0883120313C0000630C002031DB629F4
:10036000FF21082208220822082208008312031312
:100370003F0883120313C0000730C002031DC629C3
:10038000FF21FF21082208220822080083120313FC
:100390003F0883120313C0000830C002031DD62992
:1003A000FF21FF21FF2108220822080083120313E6
:1003B0003F0883120313C0000930C002031DE62961
:1003C000FF21FF21FF21FF210822080083120313D0
:1003D0003F0883120313C0000030C002031D080051
:1003E000FF21FF21FF21FF21FF2108005030A8003D
:1003F000A6016400A60BF929A80BF82908008312AE
:1004000003138516F621F621F6218512F621080040
:10041000831203138516F6218512F6210800870141
:100420008312031386000712BE228711BE2207170C
:10043000BE220713BE220800870183120313860021
:100440000716BE228711BE220717BE220713BE223F
:10045000080083120313AA00BE222A08831603137E
:100460008701860183120313860083120313071288
:10047000BE228711BE220717BE220713BE22831297
:100480000313AA0DAA0DAA0DAA0D2A088316031399
:100490008701860183120313860083120313071258
:1004A000BE228711BE220717BE220713BE220800F4
:1004B00083120313AA00831203138600831203130B
:1004C000071687110717BE220000071383120313B4
:1004D000AA0DAA0DAA0DAA0D831203132A088312CE
:1004E0000313860083120313071687110717BE2212
:1004F00000000713080086018030292208008601C9
:10050000C030292208008601943029220800860183
:10051000D430292208000A30292208000E3029226E
:1005200008001C3029220800183029220800860102
:100530000130292208000E30292208000C3029221F
:10054000080083160313FF3086008312031307127B
:100550008715071706080713803983120313031D35
:10056000A12A87118316031386010800A601A8019A
:100570006400A60BB82AA80BB82A0800FF30831223
:100580000313A600640083120313A60BC22A0800FB
:100590008316031387018316031300308600831626
:1005A0000313073081008312031300308B008B1775
:1005B0000800333029223230292228302922013004
:1005C0002922063029220800103083120313A700C5
:1005D000FF30582283120313A70BE82A0800831266
:1005E00003132730BB001030BA0016233C08B300B9
:1005F0000330BB00E830BA0016233C08B4000030DA
:10060000BB006430BA0016233C08B5000030BB00C4
:100610000A30BA0016233C08B6003808B7000800B4
:100620003030B307B407B507B607B7070030BC00D2
:100630000030BD00031383123B083902031D222B37
:100640003A083802031C0800031003113B08390262
:10065000B900031003113A083802B800031CB903AB
:100660000310BC0A0319BD0A1A2B080097227B222B
:100670008B22E4227F22E4228E227B229B2248309E
:100680005822413058224D305822203058222030F4
:100690005822433058225430582243305822533085
:1006A00058225330582220305822433058224F309D
:1006B00058224430582245305822523058227F2246
:1006C000203058222030582252305822613058228F
:1006D00064305822693058226F30582274305822C2
:1006E0006530582263305822683058226E305822C4
:1006F000693058226B3058226130582220305822FD
:10070000203058229E2208007F22831203132B08D8
:1007100083120313B800B901EF22102336085822C0
:10072000370858222F30582235305822303058227E
:100730002030582220305822663058223D3058222E
:100740002208582223085822240858222E305822E2
:1007500025085822483058227A3058222030582212
:100760000800831203132B0883120313B80005300B
:1007700083120313BA00DB2308000530831203132E
:10078000BA00C723380883120313AB000800831292
:1007900003133A08831203178D000000000083162C
:1007A00003170C140C18D22B831203170C08831296
:1007B0000313B8000800831603178C18DD2B83126F
:1007C0000313831203178D00831203133808831257
:1007D00003178C00831603170C15831203138B1356
:1007E0008316031755308D00AA308D008C148B179B
:1007F000831603178C18FA2BBE220C1183120313D5
:040800008B1708004A
:101000008B13831203132B0883120313AC000130DC
:10101000AC02031D242883120313E330A0008312C3
:1010200003130730A100203083120313A2003630CF
:1010300083120313A300373083120313A40030304C
:1010400083120313A500022F831203132B088312AC
:101050000313AC000230AC02031D472883120313B4
:10106000E330A00083120313FD30A100203083126F
:101070000313A200363083120313A3003930831206
:101080000313A400333083120313A500022F83122D
:1010900003132B0883120313AC000330AC02031DAF
:1010A0006A2883120313E530A0008312031306306D
:1010B000A100203083120313A200373083120313E0
:1010C000A300313083120313A400393083120313B9
:1010D000A500022F831203132B0883120313AC0005
:1010E0000430AC02031D8D2883120313E530A000E9
:1010F00083120313ED30A100203083120313A200EA
:10110000373083120313A300343083120313A40077
:10111000343083120313A500022F831203132B080C
:1011200083120313AC000530AC02031DB028E63077
:1011300083120313A00083120313D030A1002030C8
:1011400083120313A200373083120313A300373036
:1011500083120313A400303083120313A500022F5F
:10116000831203132B0883120313AC000630AC0266
:10117000031DD328E73083120313A0008312031347
:10118000AB30A100203083120313A200373083124A
:101190000313A300393083120313A40037308312E2
:1011A0000313A500022F831203132B0883120313CA
:1011B000AC000730AC02031DF628E830831203139D
:1011C000A000831203138030A10020308312031388
:1011D000A200383083120313A300323083120313AA
:1011E000A400353083120313A500022F83120313CA
:1011F00064002B0883120313AC000830AC02031DFB
:101200001A29E93083120313A000831203134F300D
:10121000A100203083120313A2003830831203137D
:10122000A300353083120313A40034308312031358
:10123000A500022F8312031364002B0883120313EB
:10124000AC000930AC02031D3E29EA3083120313BF
:10125000A000831203131C30A1002030831203135B
:10126000A200383083120313A30038308312031313
:10127000A400353083120313A500022F8312031339
:1012800064002B0883120313AC000A30AC02031D68
:101290006229EA3083120313A00083120313D530AE
:1012A000A100203083120313A200393083120313EC
:1012B000A300313083120313A400353083120313CB
:1012C000A500022F8312031364002B08831203135B
:1012D000AC000B30AC02031D8629EB3083120313E4
:1012E000A000831203139330A10020308312031354
:1012F000A200393083120313A30034308312031386
:10130000A400383083120313A500022F83120313A5
:1013100064002B0883120313AC000C30AC02031DD5
:10132000AA29EC3083120313A00083120313213087
:10133000A100203083120313A2003930831203135B
:10134000A300373083120313A40034308312031335
:10135000A500022F8312031364002B0883120313CA
:10136000AC000D30AC02031DCE29EC308312031308
:10137000A00083120313A630A1003130831203139F
:10138000A200303083120313A30030308312031302
:10139000A400303083120313A500022F831203131D
:1013A00064002B0883120313AC000E30AC02031D43
:1013B000F229ED3083120313A000831203134F3080
:1013C000A100313083120313A200303083120313C3
:1013D000A300333083120313A400353083120313A8
:1013E000A500022F8312031364002B08831203133A
:1013F000AC000F30AC02031D162AED30831203132C
:10140000A00083120313F630A100313083120313BE
:10141000A200303083120313A3003730831203136A
:10142000A400323083120313A500022F831203138A
:1014300064002B0883120313AC001030AC02031DB0
:101440003A2AEE3083120313A00083120313913063
:10145000A100313083120313A20031308312031331
:10146000A300303083120313A40039308312031316
:10147000A500022F8312031364002B0883120313A9
:10148000AC001130AC02031D5E2AEF30831203134F
:10149000A000831203132A30A100313083120313FA
:1014A000A200313083120313A300343083120313DC
:1014B000A400383083120313A500022F83120313F4
:1014C00064002B0883120313AC001230AC02031D1E
:1014D000822AEF3083120313A00083120313BD305E
:1014E000A100313083120313A200313083120313A1
:1014F000A300383083120313A4003830831203137F
:10150000A500022F8312031364002B088312031318
:10151000AC001330AC02031DA62AF0308312031373
:10152000A000831203134C30A10031308312031347
:10153000A200323083120313A3003330831203134B
:10154000A400303083120313A500022F831203136B
:1015500064002B0883120313AC001430AC02031D8B
:10156000CA2AF03083120313A00083120313D6306B
:10157000A100313083120313A2003230831203130F
:10158000A300373083120313A400333083120313F4
:10159000A500022F8312031364002B088312031388
:1015A000AC001530AC02031DEE2AF1308312031398
:1015B000A000831203135B30A100313083120313A8
:1015C000A200333083120313A300313083120313BC
:1015D000A400383083120313A500022F83120313D3
:1015E00064002B0883120313AC001630AC02031DF9
:1015F000122BF13083120313A00083120313DF3088
:10160000A100313083120313A2003330831203137D
:10161000A300363083120313A40035308312031362
:10162000A500022F8312031364002B0883120313F7
:10163000AC001730AC02031D362BF23083120313BB
:10164000A000831203135B30A10031308312031317
:10165000A200343083120313A3003130831203132A
:10166000A400333083120313A500022F8312031347
:1016700064002B0883120313AC001830AC02031D66
:101680005A2BF23083120313A00083120313D130BC
:10169000A100313083120313A200343083120313EC
:1016A000A300363083120313A400323083120313D5
:1016B000A500022F8312031364002B088312031367
:1016C000AC001930AC02031D7E2BF33083120313E0
:1016D000A000831203134630A1003130831203139C
:1016E000A200353083120313A30031308312031399
:1016F000A400343083120313A500022F83120313B6
:1017000064002B0883120313AC001A30AC02031DD3
:10171000A22BF33083120313A00083120313B730FC
:10172000A100313083120313A2003530831203135A
:10173000A300363083120313A4003730831203133F
:10174000A500022F8312031364002B0883120313D6
:10175000AC001B30AC02031DC62BF3308312031305
:10176000A00083120313F430A1003130831203135D
:10177000A200353083120313A30039308312031300
:10178000A400383083120313A500022F8312031321
:1017900064002B0883120313AC001C30AC02031D41
:1017A000EA2BF43083120313A000831203132330B7
:1017B000A100313083120313A200363083120313C9
:1017C000A300323083120313A400323083120313B8
:1017D000A500022F8312031364002B088312031346
:1017E000AC001D30AC02031D0E2CF4308312031329
:1017F000A000831203136130A10031308312031360
:10180000A200363083120313A30035308312031372
:10181000A400353083120313A500022F8312031393
:1018200064002B0883120313AC001E30AC02031DAE
:10183000322CF43083120313A000831203138C3074
:10184000A100313083120313A20036308312031338
:10185000A300373083120313A4003930831203131B
:10186000A500022F8312031364002B0883120313B5
:10187000AC001F30AC02031D562CF430831203134E
:10188000A00083120313C630A1003130831203136A
:10189000A200373083120313A300313083120313E5
:1018A000A400333083120313A500022F8312031305
:1018B00064002B0883120313AC002030AC02031D1C
:1018C0007A2CF43083120313A00083120313F03038
:1018D000A100313083120313A200373083120313A7
:1018E000A300333083120313A40038308312031390
:1018F000A500022F8312031364002B088312031325
:10190000AC002130AC02031D9E2CF5308312031372
:10191000A000831203132930A10031308312031376
:10192000A200373083120313A3003730831203134E
:10193000A400333083120313A500022F8312031374
:1019400064002B0883120313AC002230AC02031D89
:10195000C22CF53083120313A000831203135230FC
:10196000A100313083120313A20037308312031316
:10197000A300393083120313A400393083120313F8
:10198000A500022F8312031364002B088312031394
:10199000AC002330AC02031DE62CF5308312031398
:1019A000A000831203138830A10031308312031387
:1019B000A200383083120313A300333083120313C1
:1019C000A400353083120313A500022F83120313E2
:1019D00064002B0883120313AC002430AC02031DF7
:1019E0000A2DF53083120313A00083120313B130C4
:1019F000A100313083120313A20038308312031385
:101A0000A300363083120313A40032308312031371
:101A1000A500022F8312031364002B088312031303
:101A2000AC002530AC02031D2E2DF53083120313BC
:101A3000A00083120313E530A10031308312031399
:101A4000A200383083120313A3003930831203132A
:101A5000A400393083120313A500022F831203134D
:101A600064002B0883120313AC002630AC02031D64
:101A7000522DF63083120313A000831203130D308E
:101A8000A100313083120313A200393083120313F3
:101A9000A300323083120313A400383083120313DF
:101AA000A500022F8312031364002B088312031373
:101AB000AC002730AC02031D762DF63083120313E1
:101AC000A000831203133F30A100313083120313AF
:101AD000A200393083120313A3003630831203139C
:101AE000A400363083120313A500022F83120313C0
:101AF00064002B0883120313AC002830AC02031DD2
:101B00009A2DF63083120313A0008312031364305E
:101B1000A100313083120313A20039308312031362
:101B2000A300393083120313A4003530831203134A
:101B3000A500022F8312031364002B0883120313E2
:101B4000AC002930AC02031DBE2DF6308312031306
:101B5000A000831203139430A100323083120313C8
:101B6000A200303083120313A30033308312031317
:101B7000A400353083120313A500022F8312031330
:101B800064002B0883120313AC002A30AC02031D3F
:101B9000E22DF63083120313A00083120313B83032
:101BA000A100323083120313A200303083120313DA
:101BB000A300363083120313A400353083120313BD
:101BC000A500022F8312031364002B088312031352
:101BD000AC002B30AC02031D062EF630831203132B
:101BE000A00083120313E830A100323083120313E4
:101BF000A200313083120313A30030308312031389
:101C0000A400373083120313A500022F831203139D
:101C100064002B0883120313AC002C30AC02031DAC
:101C20002A2EF73083120313A000831203133930D6
:101C3000A100323083120313A20031308312031348
:101C4000A300383083120313A4003130831203132E
:101C5000A500022F8312031364002B0883120313C1
:101C6000AC002D30AC02031D4E2EF730831203134F
:101C7000A000831203138730A100323083120313B4
:101C8000A200323083120313A300353083120313F2
:101C9000A400373083120313A500022F831203130D
:101CA00064002B0883120313AC002E30AC02031D1A
:101CB000722EF73083120313A00083120313A73090
:101CC000A100323083120313A200323083120313B7
:101CD000A300393083120313A4003130831203139D
:101CE000A500022F8312031364002B088312031331
:101CF000AC002F30AC02031D962EF7308312031375
:101D0000A00083120313D130A100323083120313D9
:101D1000A200333083120313A30033308312031362
:101D2000A400363083120313A500022F831203137D
:101D300064002B0883120313AC003030AC02031D87
:101D4000BA2EF83083120313A000831203131A3043
:101D5000A100323083120313A20034308312031324
:101D6000A300313083120313A4003830831203130D
:101D7000A500022F8312031364002B0883120313A0
:101D8000AC003130AC02031DDE2EF8308312031399
:101D9000A000831203135F30A100323083120313BB
:101DA000A200353083120313A300303083120313D3
:101DB000A400333083120313A500022F83120313F0
:101DC00064002B0883120313AC003230AC02031DF5
:101DD000022FF83083120313A000831203137E3006
:101DE000A100323083120313A20035308312031393
:101DF000A300343083120313A40031308312031381
:101E0000A500022F1327831603138C1483120313C8
:101E10009101831203131215831203131030BE00B5
:101E20008B178A11DE28831603138512831203137E
:101E30008516202785120800553083120313A6004B
:0C1E4000640083120313A60B202F08007F
:00000001FF
